:060000000A128A11122809
:10000800FE00030EF1000408F2000A08F300831250
:1000180003137F08F4000A128A11A1280A128A1110
:10002800C128831203132C082B0403191C281D282C
:100038005328B0010314B00D2D2801300310AB0D67
:10004800AC0DFF3E031D22280130AF002F08B0077A
:100058002D28AC1F302831282128332833282C0894
:100068002E02031D39282B082D02031C3C283D288D
:1000780044282B08AD022C08031CAE03AE0244280A
:1000880001300310AC0CAB0CFF3E031D45280130BA
:10009800B002031D502851283328532853282E080E
:1000A800AC01AC072D08AB01AB075A28080001309A
:1000B800F5070318F60A0030F60701307606031D27
:1000C8006728F4307506031D6A286B287E28F50119
:1000D800F6010130F7070318F80A0030F8070A306C
:1000E80077067804031D79287A287E28F701F80115
:1000F8007E287E2808000A3083120313AB000030E4
:10010800AC007808AE01AE077708AD01AD070A125A
:100118008A1115200A128A11831203132C08B301BD
:10012800B3072B08B201B2073208203E84008313BC
:100138000008B100310786000800FB30F0007008A5
:100148008B050130B4070318B50A0030B5070A1249
:100158008A115B200A128A118330F000700883121A
:10016800031381077408FF0073088A00720884006B
:10017800710E8300FE0E7E0E0900F501F601F701EF
:10018800F801B401B50183132B30FD000130FE00E6
:100198000D30FF00203084000A128A11DD200A1277
:1001A8008A1183010A128A11FD287E088A007F08B5
:1001B80082000A128A11D9200A128A118000840A40
:1001C80004087D0603190034FF0A0319FE0ADD2816
:1001D800013083120313AB002B0883160313860523
:1001E80044308100A4308B008330831203138100D4
:1001F80008000A128A11EC200A128A1103290A122D
:100208008A117F200A128A11032903290A128A11E6
:1002180012283F3406345B344F3466346D347D34F1
:0802280027347F346F340034E9
:02400E0032FF7F
:00000001FF
